:100000000C94F3000C940E010C940E010C940E0150
:100010000C940E010C940E010C940A170C940E0112
:100020000C940E010C940E010C94D7160C94981697
:100030000C9490110C940E010C940E010C940E0172
:100040000C940E010C943B040C940E010C94511072
:100050000C94A4100C940E010C940E010C940E013F
:100060000C940E010C940E010C940E010C940E01D4
:100070004570692D4F5344205665722E302E382E10
:10008000322E340000416B7475656C6C65732053BF
:10009000657474696E67000053657474696E6720D7
:1000A000200000486F6568656E73656E736F72201F
:1000B00000004853206D697420536368616C746557
:1000C0007220000048656164696E6720486F6C6447
:1000D0002000004B6F6D706173732000004B6F6DDB
:1000E0007061737320666978200000475053204187
:1000F0006B74697620000041636873656E6B6F7086
:1001000070656C756E67200000447265687261747A
:100110006520626567722E2000004665686C657216
:100120002046433C2D3E4F5344200000556E7465DD
:10013000727370616E6E756E672000004B65696E3C
:10014000652053657474696E672D416E7A656967C1
:1001500065000050432F4254206973742065696E16
:100160006765736368616C746574000055656265EA
:10017000726E65686D65204C65747A746573205382
:10018000657474696E6700004F4E00002D2D2D00C0
:10019000004550492D4D656E750050616C0050430F
:1001A0002F4254004B656E6E756E670052432D42B0
:1001B000657472696562000045786974004F4E008D
:1001C0002D2D0076767D76767A76767E76767776C3
:1001D000767B76767876767C76767976767D7676A8
:1001E0007A76767E760011241FBECFEFD4E0DEBF94
:1001F000CDBF11E0A0E0B1E0E6ECF1E302C0059074
:100200000D92AE34B107D9F713E0AEE4B1E001C00E
:100210001D92AB3AB107E1F70C941B010C9400005E
:1002200080E981BB8FE084BBAC9AAD9A8EE28ABB39
:10023000D99ADD9A08951F93109295011092910119
:1002400010929601A0E0B0E00E94CF18802D99276F
:1002500080935501A1E0B0E00E94CF18802D99272E
:1002600080930001A2E0B0E00E94CF18802D992772
:1002700080935601A7E1B0E00E94CF18802D992706
:1002800080936D01A8E1B0E00E94CF18802D9927DE
:10029000809380010E943D160E9410010E942B0451
:1002A00080915501813019F40E943C1002C00E94D7
:1002B0002C107894A89A0E94C1030E949C040E946A
:1002C000A3088091800185FF02C00E9475130E94DF
:1002D000EB08809150018130B1F41092500180916F
:1002E0009501882351F480915501882331F4809140
:1002F0006201813011F40E9446110E9483110E9414
:1003000088110E9439148091540190919501813097
:1003100061F4992351F40E940A0E8091800185FFB7
:1003200004C00E9414130E947D13809153018130F8
:10033000B9F580919501882399F5AA9A0E943C0FFE
:1003400080916D018823A9F40E9401080E94F106A2
:100350008091800180FF04C00E9403120E948209E4
:100360008091800183FF02C00E94C8170E945B0930
:1003700016C080910201823054F00E94AB080E94A6
:1003800003120E9482090E947F0A0E945B098091E9
:100390000201833024F00E9401080E94F106AA980D
:1003A00080914E018130C1F5809195018823A1F59E
:1003B00010924E0180916D01882321F080910201FD
:1003C000833014F00E94320980916A0190916B0190
:1003D000019690936B0180936A0180916A019091DC
:1003E0006B01CC9769F48091680190916901019645
:1003F000909369018093680110926B0110926A01D9
:100400000E94E10A0E94200980915B01813021F461
:100410000E94950B0E94210D10914F01113009F09F
:1004200058CF80919501882309F053CF10924F0146
:100430000E94AB0880918601813019F0823059F416
:1004400006C00E947D0982E08093860104C00E945C
:1004500056091093860180916D01813009F039CFE2
:1004600080919501882309F034CF80916C0181300F
:1004700009F02FCF10926C0180910201813071F050
:1004800082301CF4882339F024CF823081F083300D
:1004900009F01FCF15C00E947D091BCF0E9456098D
:1004A00064E084E00E946D020E949D0412CF0E94CD
:1004B000560964E084E00E946D020E94A30807CF01
:1004C0000E94560964E084E00E946D020E94A30825
:1004D0000E94EB080E943209FCCE482FD99827E0F1
:1004E00030E0DB98000000000000000081E090E0B8
:1004F000022E02C0880F991F0A94E2F7842311F09C
:10050000DA9A01C0DA980000000000000000DB9ACF
:100510000000000000000000215030408FEF2F3F0E
:100520003807F9F627E030E0DB9800000000000013
:10053000000081E090E0022E02C0880F991F0A940B
:10054000E2F7862311F0DA9A01C0DA980000000081
:1005500000000000DB9A00000000000000002150B5
:1005600030408FEF2F3F3807F9F6DB98DA98D99AA9
:10057000089564E084E00E946D026CE480E00E94D3
:100580006D0210925001809150018823E1F36AE0DE
:100590008CE60E946D0260E085E00E946D02089585
:1005A0001F93CF93DF9380914E018823E1F3109244
:1005B0004E010E94F81010E00DC08091530181306F
:1005C00011F40E943C0F80914E01813019F4109279
:1005D0004E0111E09091810180E0112309F481E046
:1005E000992311F4882349F7C8E1D0E0882309F45E
:1005F000B1C080918F038093800180918001DE01E2
:10060000082E0E94D71845E850E061E082E00E9481
:10061000350D48E950E062E082E00E94350D43EA82
:1006200050E064E082E00E94350D42EB50E065E06E
:1006300082E00E94350D44EC50E066E082E00E94CA
:10064000350D43ED50E067E082E00E94350D4DED41
:1006500050E068E082E00E94350D4BEE50E069E02A
:1006600082E00E94350D47EF50E06AE082E00E9490
:10067000350D4CE251E06BE082E00E94350D409177
:100680007E0150917F0162E084E10E94F60C80912E
:10069000800180FF03C048E851E002C04CE851E00F
:1006A00064E084E10E94350D8091800181FF03C0E8
:1006B00048E851E002C04CE851E065E084E10E9466
:1006C000350D8091800182FF03C048E851E002C0EF
:1006D0004CE851E066E084E10E94350D8091800194
:1006E00083FF03C048E851E002C04CE851E067E0F6
:1006F00084E10E94350D8091800184FF03C048E8A9
:1007000051E002C04CE851E068E084E10E94350D00
:100710008091800185FF03C048E851E002C04CE8A9
:1007200051E069E084E10E94350D8091800186FFEF
:1007300003C048E851E002C04CE851E06AE084E1BF
:100740000E94350D40919F0355276BE084E10E9484
:10075000F60C13C045E850E062E082E00E94350DDF
:100760004AE151E065E082E00E94350DDE010E9421
:10077000CF18802D992780938001DF91CF911F9111
:1007800008950E94B90210924E0180914E01882373
:10079000E1F340E750E062E087E00E94350D0E94FF
:1007A0009D0410924E0180914E018823E1F3109236
:1007B0004E0180914E018823E1F310924E0164E0D6
:1007C00084E00E946D026CE480E00E946D028091E2
:1007D0005501882319F40E94D0021AC04CE351E05D
:1007E00062E082E00E94350D43E551E064E082E082
:1007F0000E94350D4CE651E066E082E00E94350D26
:10080000A8E1B0E00E94CF18802D99278093800145
:1008100080914E018823E1F310924E0180914E01A8
:100820008823E1F310924E0180914E018823E1F379
:1008300010924E0180914E018823E1F310924E01F7
:1008400080914E018823E1F310924E0164E084E030
:100850000E946D02089582E083BF92E49EBD8EE106
:1008600089BF83E087BD86E982BD90938A0080E2DC
:1008700080937D0008951F920F920FB60F9211245E
:100880008F939F93809152018F5F8093520180914B
:100890005201883439F591E0909351011092520140
:1008A0008091A3038F5F8093A3038091A303843679
:1008B00031F41092A30390934E0190934F018091D5
:1008C000A303823311F490934F018091A2038F5FB1
:1008D0008093A2038091A2038A3021F41092A20394
:1008E000909350019F918F910F900FBE0F901F908A
:1008F0001895282F80538A3010F090E005C02033DF
:1009000011F49AE001C0982F822F81548A3110F49B
:10091000922F9653822F81568A3110F4922F9C5336
:100920002D3211F499E403C02E3209F491E4892F99
:10093000992787FD90950895089560E085E00E94CD
:100940006D0263E886E00E946D0260E987E00E9424
:100950006D0260E085E00E946D0264E886E00E941E
:100960006D0261E987E00E946D0260E085E00E940F
:100970006D0265E886E00E946D0262E987E00E94F0
:100980006D0260E085E00E946D0266E886E00E94EC
:100990006D0263E987E00E946D0260E085E00E94DD
:1009A0006D0267E886E00E946D0264E987E00E94BC
:1009B0006D0260E085E00E946D0268E886E00E94BA
:1009C0006D0265E987E00E946D0260E085E00E94AB
:1009D0006D0269E886E00E946D0266E987E00E9488
:1009E0006D0260E085E00E946D026AE886E00E9488
:1009F0006D0267E987E00E946D0260E085E00E9479
:100A00006D0261EA86E00E946D0268E987E00E945B
:100A10006D0260E085E00E946D0262EA86E00E945D
:100A20006D0269E987E00E946D0260E085E00E9446
:100A30006D0263EA86E00E946D026AE987E00E9427
:100A40006D0260E085E00E946D0264EA86E00E942B
:100A50006D026BE987E00E946D0260E085E00E9414
:100A60006D0265EA86E00E946D026CE987E00E94F3
:100A70006D0260E085E00E946D0266EA86E00E94F9
:100A80006D026DE987E00E946D0260E085E00E94E2
:100A90006D0267EA86E00E946D026EE987E00E94BF
:100AA0006D0260E085E00E946D0268EA86E00E94C7
:100AB0006D026FE987E00E946D0260E085E00E94B0
:100AC0006D026FEB86E00E946D0260EA87E00E9493
:100AD0006D0260E085E00E946D0260EC86E00E949D
:100AE0006D0261EA87E00E946D0260E085E00E948D
:100AF0006D0261EC86E00E946D0262EA87E00E946E
:100B00006D0260E085E00E946D0262EC86E00E946A
:100B10006D0263EA87E00E946D0260E085E00E945A
:100B20006D0263EC86E00E946D0264EA87E00E9439
:100B30006D0260E085E00E946D0264EC86E00E9438
:100B40006D0265EA87E00E946D0260E085E00E9428
:100B50006D0265EC86E00E946D0266EA87E00E9405
:100B60006D0260E085E00E946D0266EC86E00E9406
:100B70006D0267EA87E00E946D0260E085E00E94F6
:100B80006D026DED86E00E946D0268EA87E00E94CA
:100B90006D0260E085E00E946D026EED86E00E94CD
:100BA0006D0269EA87E00E946D0260E085E00E94C4
:100BB0006D026FED86E00E946D026AEA87E00E9496
:100BC0006D0260E085E00E946D0260EE86E00E94AA
:100BD0006D026BEA87E00E946D0260E085E00E9492
:100BE0006D0261EE86E00E946D026CEA87E00E9471
:100BF0006D0260E085E00E946D0262EE86E00E9478
:100C00006D026DEA87E00E946D0260E085E00E945F
:100C10006D0263EE86E00E946D026EEA87E00E943C
:100C20006D0260E085E00E946D0264EE86E00E9445
:100C30006D026FEA87E00E946D0260E085E00E942D
:100C40006D026BEF86E00E946D0260EB87E00E9410
:100C50006D0260E085E00E946D026CEF86E00E940C
:100C60006D0261EB87E00E946D0260E085E00E940A
:100C70006D026DEF86E00E946D0262EB87E00E94DC
:100C80006D0260E085E00E946D026EEF86E00E94DA
:100C90006D0263EB87E00E946D0260E085E00E94D8
:100CA0006D026FEF86E00E946D0264EB87E00E94A8
:100CB0006D0261E085E00E946D0260E086E00E94C6
:100CC0006D0265EB87E00E946D0261E085E00E94A5
:100CD0006D0261E086E00E946D0266EB87E00E9493
:100CE0006D020895FF920F931F93CF93DF938C01B2
:100CF000F62EEC0117C06D2F772785E00E946D025C
:100D00006C2F86E00E946D028F2D9927FC01EE0F5B
:100D1000FF1FE80FF91FE15FFE4F608187E00E942F
:100D20006D022196C8010596C817D90720F3E8017E
:100D30002A9617C06D2F772785E00E946D026C2FD1
:100D400086E00E946D028F2D9927FC01EE0FFF1F98
:100D5000E80FF91FE15FFE4F608187E00E946D029E
:100D60002196C8010F96C817D90720F3DF91CF91BC
:100D70001F910F91FF9008950F931F93CF93DF93CF
:100D80008C01EC010EC06D2F772785E00E946D026B
:100D90006C2F86E00E946D0260E087E00E946D0289
:100DA0002196C8010596C817D90768F3E8012A9665
:100DB0000EC06D2F772785E00E946D026C2F86E0B4
:100DC0000E946D0260E087E00E946D022196C801DA
:100DD0000F96C817D90768F3DF91CF911F910F9134
:100DE00008951F93CF93DF93809143039091440321
:100DF00066E170E00E949A189B012E5F3F4F37FD1D
:100E00001BC0C9016AE070E00E949A18182F16955D
:100E1000C9016AE070E00E949A1887E090E0861BA2
:100E200091092EE130E0829FE001839FD00D929FD7
:100E3000D00D1124279616C0309521953F4FC9013A
:100E40006AE070E00E949A18182F16951C5FC9017D
:100E50006AE070E00E949A188EE1689FE001112418
:100E6000C950DF4F80910B0190910C01C817D90731
:100E700039F080910B0190910C010E94BC0604C0D6
:100E800080918401811721F0612FCE010E947206AA
:100E900010938401D0930C01C0930B01DF91CF918B
:100EA0001F910895AF92BF92DF92EF92FF920F933E
:100EB0001F93CF93DF93CDB7DEB721970FB6F8948A
:100EC000DEBF0FBECDBF8C01D62E5C0119826B2D0B
:100ED000772785E00E946D026A2D86E00E946D02F0
:100EE000ED2CFF24F701E35DFE4F608187E00E9457
:100EF0006D028EE190E0A80EB91E9981925E9983F1
:100F00009C3329F7F4EBAF2EB12CA00EB11E6B2D44
:100F1000772785E00E946D026A2D86E00E946D02AF
:100F2000F701E35DFE4F608187E00E946D02EEE114
:100F3000F0E0AE0EBF1EC801825F9E4FA816B90634
:100F400031F721960FB6F894DEBF0FBECDBFDF910B
:100F5000CF911F910F91FF90EF90DF90BF90AF90D6
:100F60000895EF92FF920F931F93CF93DF93CDB726
:100F7000DEB721970FB6F894DEBF0FBECDBF8C0150
:100F80007C0119826F2D772785E00E946D026E2DFE
:100F900086E00E946D0260E087E00E946D028EE1B3
:100FA00090E0E80EF91E9981925E99839C3351F787
:100FB00084EBE82EF12CE00EF11E6F2D772785E0F3
:100FC0000E946D026E2D86E00E946D0260E087E057
:100FD0000E946D02EEE1F0E0EE0EFF1EC801825F9E
:100FE0009E4FE816F90649F721960FB6F894DEBF32
:100FF0000FBECDBFDF91CF911F910F91FF90EF906A
:1010000008951F93CF93DF938091450390914603FA
:1010100066E170E00E949A189B012A5F3F4F37FDFE
:1010200012C0C9016AE070E00E949A18182F169544
:101030001C5FC9016AE070E00E949A18C6E8D0E01F
:10104000C61BD10913C0309521953F4FC9016AE0F5
:1010500070E00E949A18182F1695C9016AE070E096
:101060000E949A18C62FDD27C957DF4F80910D01C6
:1010700090910E01C817D90739F080910D01909118
:101080000E010E94B10704C080918501811721F0F3
:10109000612FCE010E94520710938501D0930E015B
:1010A000C0930D01DF91CF911F91089560E085E01D
:1010B0000E946D026FEC86E00E946D026CE887E092
:1010C0000E946D0261E085E00E946D026BE086E0A7
:1010D0000E946D026DE887E00E946D020895EF9214
:1010E000FF920F931F93CF93DF937A019EE1699F45
:1010F000B0011124680F711D8B01020F111D109298
:10110000A403EB0116C06D2F772785E00E946D02C6
:101110006C2F86E00E946D028091A403F701E80F16
:10112000F11D60818F5F8093A40387E00E946D02B0
:101130002196C017D10738F3DF91CF911F910F91FE
:10114000FF90EF90089525E046E051E06EE081E0E9
:101150000E946F080895CF93DF93CDB7DEB7249731
:101160000FB6F894DEBF0FBECDBF19821A8285E498
:101170008B831C82F894789430915503832F6AE016
:101180000E947A18282F0E947A18482F822F0E94D6
:101190007A18292F832F0E947A18992319F48AE04C
:1011A0008C8301C09C83222319F48AE08A8301C0C6
:1011B0002A83498324E0AE014F5F5F4F61E083E003
:1011C0000E946F0824960FB6F894DEBF0FBECDBF05
:1011D000DF91CF910895CF93DF93CDB7DEB72497FA
:1011E0000FB6F894DEBF0FBECDBF80E28A839BE0CE
:1011F000998381E38B839C8321E0AE014E5F5F4F37
:1012000061E081E00E946F0880915B01813079F498
:1012100021E0AE014F5F5F4F62E00E946F0822E065
:10122000AE014D5F5F4F63E081E00E946F0824963E
:101230000FB6F894DEBF0FBECDBFDF91CF910895FA
:1012400080915601813069F42091A301922F27FDEE
:101250009F5F959544EA51E061E08EE0891B0E9412
:101260006F080895CF93DF93CDB7DEB725970FB6FC
:10127000F894DEBF0FBECDBFDE011196EAE3F1E0C8
:1012800085E001900D928150E1F725E0AE014F5FBE
:101290005F4F67E08CE00E946F0825960FB6F894C8
:1012A000DEBF0FBECDBFDF91CF9108956CE480E02B
:1012B0000E946D0208958091570390915803843BDA
:1012C000910554F080919F03992720915503309107
:1012D00056038217930744F080918601882361F4B6
:1012E00081E080938601089580918601181614F498
:1012F0000E94560910928601089562E480E00E94DF
:101300006D020895EF92FF920F931F93CF93DF9397
:10131000CDB7DEB72F970FB6F894DEBF0FBECDBFA7
:1013200085E0FE01369611928A95E9F780914D038A
:1013300090914E036EE170E00E949A18CB018E01ED
:10134000055F1F4F019797FF02C080E090E04AE0E1
:1013500050E0B8010E941518F80101900020E9F74B
:101360003197EE2EE01A1092A403FF240AC00E0F4C
:101370001F1FEC0FFD1F83850E947904F8018083F5
:10138000F394EF2DFF278E2D992787FD90958E01E1
:101390000F5F1F4FE817F90754F3F092A40325E0FD
:1013A000AE014A5F5F4F69E085E10E946F082E2D14
:1013B000A80169E089E18E190E946F082F960FB687
:1013C000F894DEBF0FBECDBFDF91CF911F910F917B
:1013D000FF90EF900895EF92FF920F931F93CF939A
:1013E000DF93CDB7DEB72E970FB6F894DEBF0FBEF2
:1013F000CDBF19821A821B821C8280917601909146
:1014000077018E01065F1F4F4AE050E0B8010E944D
:101410001518F80101900020E9F73197EE2EE01A37
:101420001092A403FF240AC00E0F1F1FEC0FFD1F14
:1014300082850E947904F8018083F394EF2DFF27C1
:101440008E2D992787FD90958E010B5F1F4FE81712
:10145000F90754F3F092A40324E0AE014F5F5F4F0D
:1014600066E085E10E946F082E2DA80166E089E103
:101470008E190E946F08809176019091770118165D
:10148000190664F460E085E00E946D0262EC86E07B
:101490000E946D026CE887E00E946D0280917601E7
:1014A0009091770197FF0CC060E085E00E946D028B
:1014B00062EC86E00E946D026DE887E00E946D029A
:1014C0008091760190917701892B61F460E085E04D
:1014D0000E946D0262EC86E00E946D0260E087E08F
:1014E0000E946D022E960FB6F894DEBF0FBECDBFE0
:1014F000DF91CF911F910F91FF90EF900895EF92A0
:10150000FF920F931F93CF93DF93CDB7DEB72B9747
:101510000FB6F894DEBF0FBECDBFDE011196E7E334
:10152000F1E083E001900D928150E1F78E01085FB8
:101530001F4F4AE050E0B80180915303909154034B
:101540000E941518F80101900020E9F73197EE2E5E
:10155000E01A1092A403FF240AC00E0F1F1FEC0F05
:10156000FD1F80850E947904F8018083F394EF2D9C
:10157000FF278E2D992787FD90958E010C5F1F4FB9
:10158000E817F90754F3F092A40323E0AE014F5F8C
:101590005F4F6EE08DE00E946F082E2DA8016EE077
:1015A00080E18E190E946F082B960FB6F894DEBF6B
:1015B0000FBECDBFDF91CF911F910F91FF90EF90A4
:1015C0000895EF92FF920F931F93CF93DF93CDB7C0
:1015D000DEB728970FB6F894DEBF0FBECDBF1982D5
:1015E0008AE08A8380916801909169018E010A5F87
:1015F0001F4F4AE050E0B8010E941518F801019011
:101600000020E9F73197EE2EE01A1092A403FF2490
:101610000DC08E010D5F1F4F0E0F1F1FEC0FFD1F22
:1016200086810E947904F8018083F394EF2DFF27CF
:101630008E2D992787FD9095E817F90754F3F092BE
:10164000A40380916801909169018E010D5F1F4F85
:101650000A976CF421E0AE014F5F5F4F6EE081E0CE
:101660000E946F0821E0A8016EE082E004C022E041
:10167000A8016EE081E00E946F0880916A0190915C
:101680006B018E010A5F1F4F4AE050E0B8010E94D3
:101690001518F80101900020E9F73197EE2EE01AB5
:1016A0001092A403FF240DC08E010D5F1F4F0E0F7B
:1016B0001F1FEC0FFD1F86810E947904F8018083B3
:1016C000F394EF2DFF278E2D992787FD9095E8172E
:1016D000F90754F3F092A40380916A0190916B0191
:1016E0008E010D5F1F4F0A976CF421E0AE014E5F33
:1016F0005F4F6EE084E00E946F0821E0A8016EE079
:1017000085E004C022E0A8016EE084E00E946F083A
:1017100028960FB6F894DEBF0FBECDBFDF91CF91F4
:101720001F910F91FF90EF900895CF92DF92EF926B
:10173000FF920F931F93CF93DF93CDB7DEB72B9715
:101740000FB6F894DEBF0FBECDBF80915C019091C3
:101750005D0180915C0190915D018D5A964230F05F
:101760008CEA96E290935D0180935C0180915C012C
:1017700090915D0164E670E00E94861870935801B4
:101780006093570180915C0190915D0164E670E087
:101790000E94861890935A018093590180915901B3
:1017A00090915A016AE070E00E94861870935A0185
:1017B00060935901809157019091580125E4298344
:1017C0001A821B828E01085F1F4F4AE050E0B80169
:1017D0000E941518F80101900020E9F73197CE2EEC
:1017E000C01A1092A403DD240BC0020F131FE20ED7
:1017F000F31EF70180810E947904F8018083D3945D
:101800002D2D33278C2D992787FD909548E0E42EC8
:10181000F12CEC0EFD1E8E010C5F1F4F28173907AF
:1018200024F3D092A40322E0AE014E5F5F4F62E04A
:1018300083E00E946F082C2DA80162E085E08C19DE
:101840000E946F088091590190915A014AE050E03E
:10185000B7010E941518F70101900020E9F73197B0
:10186000EE19EE2E1092A403FF240AC00E0F1F1FC4
:10187000EC0FFD1F80850E947904F8018083F394AA
:10188000EF2DFF278E2D992787FD90958E010C5FF8
:101890001F4FE817F90754F3F092A40321E0AE01BB
:1018A0004F5F5F4F62E085E00E946F0821E0AE016C
:1018B0004E5F5F4F62E086E00E946F0821E0A80162
:1018C00062E086E00E946F082B960FB6F894DEBFA8
:1018D0000FBECDBFDF91CF911F910F91FF90EF9081
:1018E000DF90CF9008950F931F93CF93DF93CDB7E1
:1018F000DEB72A970FB6F894DEBF0FBECDBF4AE021
:1019000050E08E010F5F1F4FB8010E941518F801BB
:1019100001900020E9F73197E01B1092A40320E02A
:10192000FF27E7FDF09501C02F5F822F99278E17C3
:101930009F07D4F32093A4032A960FB6F894DEBF32
:101940000FBECDBFDF91CF911F910F9108959F9250
:10195000AF92BF92CF92DF92EF92FF920F931F93BD
:10196000CF93DF93CDB7DEB76E970FB6F894DEBF97
:101970000FBECDBF982EA62E7A01FA01019000204D
:10198000E9F73197BE2EB41ACC24DD240BC0FF2713
:101990008A010E0F1F1FEE0DFF1D80810E9479042A
:1019A000F8018083EC2D0894C11CD11C8B2D992744
:1019B0000196AE014F5F5F4FC816D90641F72B2D38
:1019C0006A2D892D0E946F086E960FB6F894DEBFBF
:1019D0000FBECDBFDF91CF911F910F91FF90EF9080
:1019E000DF90CF90BF90AF909F900895EF92FF92BD
:1019F0000F931F93CF93DF93CDB7DEB764970FB6E6
:101A0000F894DEBF0FBECDBFE82EF62ECA014AE025
:101A100050E08E010F5F1F4FB8010E941518A801FA
:101A20006F2D8E2D0E94A70C64960FB6F894DEBF22
:101A30000FBECDBFDF91CF911F910F91FF90EF901F
:101A4000089560915E0170915F01809160019091B5
:101A5000610128E631E040E050E00E94AD18A901A4
:101A600063E083E00E94F60C0895BF92CF92DF926C
:101A7000EF92FF920F931F93CF93DF93CDB7DEB713
:101A800064970FB6F894DEBF0FBECDBFB82EC62E3A
:101A90009A01DE01119605C0EA0FFB1F90832F5FAC
:101AA0003F4F822F841BF9019491E82FFF27992340
:101AB00099F7EA0FFB1F1082FD0101900020E9F762
:101AC0003197DE2EDA1AEE24FF2409C08D01020FB1
:101AD000111DF80180810E947904F80180832E2D68
:101AE0000894E11CF11C8D2D99270196DE011196B9
:101AF000E816F90659F72D2DAD016C2D8B2D0E949E
:101B00006F0864960FB6F894DEBF0FBECDBFDF91AD
:101B1000CF911F910F91FF90EF90DF90CF90BF90EA
:101B20000895EF92FF920F931F93CF93DF9333E0CB
:101B3000E32EF12CC0E0D0E0AEEAB2E08C91FD01E2
:101B4000218112810381B7016C5F7F4F7B01149665
:101B5000F2E0633D7F0709F456C0422F55274D53ED
:101B60005040E0914301F0914401EC0FFD1F992793
:101B7000CD97880F991F880F991F9A01689413F8C1
:101B8000359527951694E1F7822B932B8083673246
:101B90007105C9F1212F33272D533040FE013196B5
:101BA0008091430190914401E80FF91F4F705070EC
:101BB00084E0440F551F8A95E1F7C90195958795F3
:101BC00095958795482B592B408381E06B37780793
:101BD000D1F0FE0132968091430190914401E80FCB
:101BE000F91F2370307086E0220F331F8A95E1F7CA
:101BF000802F9927CD97282B392B20836F5C72403B
:101C000011F023969BCFDF91CF911F910F91FF9001
:101C1000EF9008952F923F924F925F926F927F9232
:101C20008F929F92AF92BF92CF92DF92EF92FF92EC
:101C30000F931F93CF93DF938091BA01843469F09F
:101C4000A1E4B0E060E070E053E0C52ED12C8DC07F
:101C5000B8018BC0AFEFBFEF88C060E070E043E039
:101C6000C42ED12C32E0A32EB12C01E010E020E4F0
:101C7000222E312C9FE3492E512CCBEBD1E08EE369
:101C8000682E712C888129819A808B8044E050E0F5
:101C9000C40ED51E24967B01D101A61BB70B61345F
:101CA000710509F462C0422F55274D535040E09111
:101CB0004101F0914201E60FF71F9927CD97880F58
:101CC000991F880F991F9A01A4E035952795AA9529
:101CD000E1F7822B932B8083D201A61BB70B6034D4
:101CE000710509F4B5CF292D33272D533040E091EC
:101CF0004101F0914201E00FF11F4F70507074E00C
:101D0000440F551F7A95E1F7C901959587959595EB
:101D10008795482B592B4083B501D301AE19BF09D4
:101D20005BE5C516D10409F495CFE0914101F0912E
:101D30004201EA0DFB1D2370307096E0220F331F25
:101D40009A95E1F7882D9927CD97282B392B208359
:101D5000B7016D5F7F4F83E090E0A80EB91E0D5F65
:101D60001F4F6134710509F08DCF8091BA01813523
:101D700009F06DC069C0F601E854FE4F2081F601FC
:101D8000E754FE4F8081F601E654FE4F1081F601C4
:101D9000E554FE4F0081482F55274D535040E091A8
:101DA0004501F0914601E60FF71F33272D533040D0
:101DB000220F331F220F331FCA01689413F8959521
:101DC00087951694E1F7282B392B2083A130B10594
:101DD000F1F1212F33272D533040FB0131968091B3
:101DE000450190914601E80FF91F4F70507084E053
:101DF000440F551F8A95E1F7C901959587959595EB
:101E00008795482B592B408313979FEFAF3FB90716
:101E1000F1F044E050E0C40ED51E6E5F7F4FE091BC
:101E20004501F0914601E60FF71F2370307046E040
:101E3000220F331F4A95E1F7802F9927CD97282B42
:101E4000392B20836F5F7F4F109709F094CF10924A
:101E50005401DF91CF911F910F91FF90EF90DF9090
:101E6000CF90BF90AF909F908F907F906F905F903A
:101E70004F903F902F900895EF92FF920F931F93F2
:101E8000CF93DF938091AD02843409F091C033E0A9
:101E9000E32EF12C60E070E0AEEAB2E08C91FD013F
:101EA000218112810381E70124967E011496613419
:101EB000710509F456C0422F55274D535040E0910B
:101EC0003F01F0914001E60FF71F9927CD97880F4A
:101ED000991F880F991F9A01689413F835952795D3
:101EE0001694E1F7822B932B808360347105C9F13E
:101EF000212F33272D533040FB01319680913F0134
:101F000090914001E80FF91F4F70507084E0440F2A
:101F1000551F8A95E1F7C901959587959595879500
:101F2000482B592B4083CB35D105D9F0FB01329694
:101F300080913F0190914001E80FF91F23703070AC
:101F400016E0220F331F1A95E1F7802F9927CD97BE
:101F5000282B392B20836E33710519F06D5F7F4F6D
:101F60009DCF8091570390915803843B91058CF449
:101F7000809162018130E1F410926201F8940E9434
:101F80003C1078948091570390915803843B9105BD
:101F90007CF080916201882359F481E08093620192
:101FA000F89480915501882311F40E942C107894A4
:101FB0008091AD028C3459F481E090E090937F01E0
:101FC00080937E0181E0809381010E94910D809138
:101FD000AD028D3459F482E090E090937F018093BC
:101FE0007E0181E0809381010E94910D8091AD027C
:101FF0008E3459F483E090E090937F0180937E01CA
:1020000081E0809381010E94910D8091AD028F3417
:1020100059F484E090E090937F0180937E0181E009
:10202000809381010E94910D8091AD02803559F419
:1020300085E090E090937F0180937E0181E0809322
:1020400081010E94910D10925301DF91CF911F9158
:102050000F91FF90EF90089582E289B910BC80B98A
:102060001CBE909A28E92AB996E890BD82EC8BB9FB
:1020700021B99CBF82B9089582E289B910BC80B9A8
:102080001CBE909A88E98AB926E820BD92EC9BB9DB
:1020900080E981B92CBF92B90895159BFECF83B911
:1020A00008951F920F920FB60F9211248F939F9352
:1020B000EF93FF939CB19093A5039D3081F48091A1
:1020C0008801813061F4AB981092880180935401AB
:1020D000E0918603FF27E854FE4F90832CC0809147
:1020E0008801882319F0813031F513C0933239F417
:1020F00080915401882319F481E080938801109223
:10210000860380918603E82FFF27E854FE4F9083D3
:102110000CC0E0918603FF27E854FE4F9083809126
:102120008603853930F4809186038F5F8093860320
:1021300002C010928801FF91EF919F918F910F90B3
:102140000FBE0F901F9018951F920F920FB60F920F
:1021500011248F939F93EF93FF9393B19093A603D2
:102160009D3081F480918701813061F4AB981092A9
:10217000870180935301E0918303FF27E555FD4FCD
:1021800090832DC080918701882319F0813039F523
:1021900014C0933241F480915301882321F481E0EB
:1021A00080938701AB9A1092830380918303E82F79
:1021B000FF27E555FD4F90830CC0E0918303FF2777
:1021C000E555FD4F908380918303853930F48091EC
:1021D00083038F5F8093830302C010928701FF9176
:1021E000EF919F918F910F900FBE0F901F901895B8
:1021F000CF93DF93CDB7DEB72C970FB6F894DEBF41
:102200000FBECDBF83E289831A8281E78B838CE77F
:102210008C838DE68D838DE38E838F8320E030E089
:10222000FE013196AE01485F5F4F8191280F311D4D
:10223000E417F507D1F7C90160E070E10E949A1830
:102240009C0160E470E00E949A18635C6887C90191
:1022500060E470E00E949A18835C89878DE08A8729
:10226000FE0131969E01255F3F4F8081159BFECF79
:1022700083B93196E217F307C1F72C960FB6F8949D
:10228000DEBF0FBECDBFDF91CF910895CF93DF9317
:10229000CDB7DEB72A970FB6F894DEBF0FBECDBF1D
:1022A00083E289831A8283E68B831C821D8286E8FF
:1022B00090E060E070E10E949A189C0160E470E098
:1022C0000E949A18635C6E83C90160E470E00E940A
:1022D0009A18835C8F838DE08887FE0131969E017A
:1022E000275F3F4F8081159BFECF83B93196E21760
:1022F000F307C1F72A960FB6F894DEBF0FBECDBF25
:10230000DF91CF91089585B392E0892785BB089529
:1023100090916501913019F485B3892785BB0895A3
:102320001F920F920FB60F9211242F933F935F933A
:102330006F937F938F939F93AF93BF938091890106
:1023400090918A01892B81F484B595B59093900181
:1023500080938F018EB58F7B8EBD81E090E090934E
:102360008A018093890141C084B595B590938E010F
:1023700080938D012EB520642EBD20918F01309168
:102380009001821B930B10928A011092890186564C
:1023900098406CE271E00E94861870938C01609303
:1023A0008B0177FF05C010928C0110928B0109C040
:1023B0006730710534F086E090E090938C01809353
:1023C0008B0120918B0130918C0180910201992722
:1023D00087FD90952817390741F0263031052CF4F8
:1023E0002093020181E080936C01BF91AF919F9196
:1023F0008F917F916F915F913F912F910F900FBEC1
:102400000F901F90189580914D0390914E039093DB
:102410006F0180936E0180916E0190916F01209108
:10242000700130917101821B930B90937301809323
:10243000720180916E0190916F0190937101809370
:10244000700140917A0150917B012091720130918D
:102450007301CA01E3E0880F991FEA95E1F7841B35
:10246000950B73E0220F331F7A95E1F7820F931FCC
:1024700068E070E00E949A1870937B0160937A0183
:1024800020917C0130917D0140917A0150917B0136
:10249000C90163E0880F991F6A95E1F7821B930BCE
:1024A000840F951F68E070E00E949A1870937D0178
:1024B00060937C0180917C0190917D0190937701E4
:1024C000809376010E94EB090895BF92CF92DF922C
:1024D000EF92FF920F931F93CF93DF93CDB7DEB7A9
:1024E00060970FB6F894DEBF0FBECDBF19821A8277
:1024F0001B821C8280918602909187029093AA038E
:102500008093A90380918802909189029093A803F7
:102510008093A7038091A9039091AA038E01055F80
:102520001F4F4AE050E0B8010E941518F8010190D1
:102530000020E9F73197BE2EB01ACC24DD240DC05F
:10254000EC0CFD1CF70180810E9479040C0D1D1D0F
:10255000F80180830894C11CD11C8B2D992787FD1D
:1025600090952BE0E22EF12CEC0EFD1E8E010B5F00
:102570001F4FC816D90624F324E0AE014F5F5F4F0A
:1025800061E08CE00E946F082B2DA80161E080E1E2
:102590008B190E946F088091A7039091A8034AE0CD
:1025A00050E0B7010E941518F70101900020E9F7EB
:1025B0003197DE2EDE18EE24FF240DC0FE01EE0D55
:1025C000FF1D83850E9479040E0D1F1DF801808375
:1025D0000894E11CF11C8D2D992787FD90958E01A3
:1025E0000B5F1F4FE816F9064CF324E0AE014F5F76
:1025F0005F4F62E08CE00E946F082D2DA80162E021
:1026000080E18D190E946F0860960FB6F894DEBFC6
:102610000FBECDBFDF91CF911F910F91FF90EF9033
:10262000DF90CF90BF900895DF92EF92FF920F93CB
:102630001F93CF93DF93CDB7DEB72B970FB6F894E8
:10264000DEBF0FBECDBFDE011196EBE4F1E083E00B
:1026500001900D928150E1F78E01085F1F4F80912C
:10266000AA024AE050E0B80199270E941518F80123
:1026700001900020E9F73197DE2ED01AEE24FF24D6
:102680000DC0FE01EE0DFF1D80850E9479040E0D28
:102690001F1DF80180830894E11CF11C8D2D9927E2
:1026A00087FD90958E010C5F1F4FE816F9064CF3DD
:1026B00023E0AE014F5F5F4F61E088E10E946F0849
:1026C0002D2DA80161E08BE18D190E946F082B96DA
:1026D0000FB6F894DEBF0FBECDBFDF91CF911F9133
:1026E0000F91FF90EF90DF90089522E049E451E0D0
:1026F00061E08AE10E946F0808956F927F928F9245
:102700009F92BF92CF92DF92EF92FF920F931F930F
:10271000CF93DF93CDB7DEB764970FB6F894DEBFE3
:102720000FBECDBF19821A821B821C826090A60246
:102730007090A7028090A8029090A9028E01035F7A
:102740001F4F6091A2027091A3028091A402909108
:10275000A5022AE030E0A8010E943618F801019095
:102760000020E9F73197BE2EB01ACC24DD240DC02D
:10277000EC0CFD1CF70180810E9479040C0D1D1DDD
:10278000F80180830894C11CD11C8B2D992787FDEB
:1027900090953DE0E32EF12CEC0EFD1E8E010B5FBB
:1027A0001F4FC816D90624F324E0AE014F5F5F4FD8
:1027B0006DE084E10E946F082B2DA8016DE088E197
:1027C0008B190E946F082AE030E0A701C401B30111
:1027D0000E943618F70101900020E9F73197DE2EAC
:1027E000DE18EE24FF240DC0FE01EE0DFF1D8585D1
:1027F0000E9479040E0D1F1DF80180830894E11CCE
:10280000F11C8D2D992787FD90958E010B5F1F4F31
:10281000E816F9064CF324E0AE014F5F5F4F6EE01F
:1028200084E10E946F082D2DA8016EE088E18D19CA
:102830000E946F0864960FB6F894DEBF0FBECDBF3E
:10284000DF91CF911F910F91FF90EF90DF90CF908C
:10285000BF909F908F907F906F900895F89488E13B
:1028600090E028E00FB6F894A89581BD0FBE21BD79
:10287000FFCF1F939D9902C1809191018F5F80933B
:10288000910191E09093930180919101853009F03D
:10289000F9C080919501882309F071C0909395014A
:1028A0001092960164E084E00E946D022091A301E1
:1028B00044EA51E061E083E00E946F0841E951E0A1
:1028C00063E083E00E94350D68E084E00E946D02C1
:1028D0004AE951E065E083E00E94350D80910001F6
:1028E000813019F44DEB51E002C040EC51E065E05D
:1028F00084E10E94350D60E084E00E946D024EE9A3
:1029000051E066E083E00E94350D809155018130F1
:1029100019F44DEB51E002C040EC51E066E084E177
:102920000E94350D44EA51E067E083E00E94350DD6
:1029300080915601813019F44DEB51E002C040EC1A
:1029400051E067E084E10E94350D4CEA51E068E017
:1029500083E00E94350D80916D01813019F44DEBBB
:1029600051E002C040EC51E068E084E10E94350D86
:1029700048EB51E06BE083E00E94350D81C010917F
:102980009601113001F568E084E00E946D028091AB
:102990005501882329F4109355014DEB51E004C0F3
:1029A0001092550140EC51E066E084E10E94350D43
:1029B00080915501A0E0B0E0082E0E94D71860E099
:1029C00084E00E946D0280919601823009F568E0F2
:1029D00084E00E946D0280915601882331F481E0E9
:1029E000809356014DEB51E004C01092560140EC2B
:1029F00051E067E084E10E94350D80915601A2E02C
:102A0000B0E0082E0E94D71860E084E00E946D02BA
:102A100080919601833009F568E084E00E946D02A0
:102A200080916D01882331F481E080936D014DEB3D
:102A300051E004C010926D0140EC51E068E084E187
:102A40000E94350D80916D01A7E1B0E0082E0E9433
:102A5000D71860E084E00E946D0280919601843076
:102A600089F410929501F89488E190E028E00FB67F
:102A7000F894A89581BD0FBE21BDFFCF10929101A2
:102A8000109293019C99E9C090919501913009F0C1
:102A9000EAC090939401809192018F5F809392019C
:102AA00080919201853009F0DEC0109292018091F0
:102AB0009601823009F464C0833030F4882359F0E1
:102AC000813009F0D0C031C0833009F483C0843034
:102AD00009F0C9C09EC0909396014AE951E065E0B3
:102AE00083E00E94350D80910001813019F44DEB97
:102AF00051E002C040EC51E065E084E10E94350DF8
:102B000068E084E00E946D024EE951E066E083E0F7
:102B10000E94350D80915501813019F44DEB51E043
:102B200002C040EC51E066E090C082E080939601E4
:102B30004EE951E066E083E00E94350D8091550139
:102B4000813019F44DEB51E002C040EC51E066E0F9
:102B500084E10E94350D68E084E00E946D0244EA41
:102B600051E067E083E00E94350D8091560181308D
:102B700019F44DEB51E002C040EC51E067E065C054
:102B800083E08093960144EA51E067E00E94350DAE
:102B900080915601813019F44DEB51E002C040ECB8
:102BA00051E067E084E10E94350D68E084E00E9416
:102BB0006D024CEA51E068E083E00E94350D80919F
:102BC0006D01813019F44DEB51E002C040EC51E051
:102BD00068E03BC084E0809396014CEA51E068E0F5
:102BE00083E00E94350D80916D01813019F44DEB29
:102BF00051E002C040EC51E068E084E10E94350DF4
:102C000068E084E00E946D0248EB51E06BE083E0F5
:102C10001DC01092960148EB51E06BE083E00E94EA
:102C2000350D68E084E00E946D024AE951E065E0FC
:102C300083E00E94350D80910001813019F44DEB45
:102C400051E002C040EC51E065E084E10E94350DA6
:102C500060E084E00E946D0206C0109292018091B3
:102C60009301809194011F910895813029F4A0E08F
:102C7000B0E0062E0E94D7180895EF92FF920F93AE
:102C80001F93CF93DF93CDB7DEB764970FB6F89459
:102C9000DEBF0FBECDBF40E050E08E010F5F1F4F83
:102CA000842F9927DC01AD5FBF4F0E94CF18202DE4
:102CB0003327F801E80FF91F20832223F1F04F5F3B
:102CC0005F4F2F3F69F7108218C0FE01E00FF11F20
:102CD00081810E9479040C551E4FF80180830E2DCE
:102CE00011270894E11CF11C8091A301992787FD0D
:102CF0009095081719074CF30EC0DE011196FD01DF
:102D000001900020E9F73197EA1BFB0BE093A30148
:102D1000EE24FF24E4CF64960FB6F894DEBF0FBE16
:102D2000CDBFDF91CF911F910F91FF90EF9008954C
:102D30001F920F920FB60F9211248F939F93809141
:102D40009A018130A1F0813018F0823049F525C018
:102D5000809198018E3129F41092980181E080933E
:102D60009A01809198018F5F8093980119C090918A
:102D70009901923061F4109299018091970181300C
:102D800019F490939A0103C083E080939A01809193
:102D900099018F5F8093990103C083E080939A012A
:102DA0009F918F910F900FBE0F901F9018951F92BB
:102DB0000F920FB60F9211248F9380919A01833056
:102DC00011F410929A018F910F900FBE0F901F90E7
:102DD0001895809143039091440365E070E00E9450
:102DE0009A1866507F4F77FD0FC081E0653F7807E6
:102DF0001CF064EF71E003C06B3F71053CF06A5F4B
:102E000081E08093970104C060E070E01092970128
:102E100062BD08951F920F920FB60F921124EF9288
:102E2000FF920F931F932F933F934F935F936F9353
:102E30007F938F939F93AF93BF93EF93FF93809173
:102E40009B01882389F48091800090918100909368
:102E5000A2018093A10180918A008F7B80938A00D8
:102E600081E080939B017FC08091800090918100E0
:102E700090935D0180935C0180918A0080648093CF
:102E80008A00109289001092880010929B01809114
:102E90005C0190915D012091A1013091A201821B02
:102EA000930B90935D0180935C0180915C01909104
:102EB0005D019695879590935D0180935C0180916B
:102EC0005C0190915D018456904090935D018093E8
:102ED0005C0180915C0190915D019C014427552724
:102EE00080919C0190919D01A0919E01B0919F01C4
:102EF000280F391F4A1F5B1F20939C0130939D01AF
:102F000040939E0150939F018091A001843130F144
:102F10001092A001E0905E01F0905F0100916001CD
:102F200010916101CA01B90124E130E040E050E0B4
:102F30000E94AD18E20EF31E041F151FE0925E0101
:102F4000F0925F01009360011093610110929C0167
:102F500010929D0110929E0110929F018091A001FC
:102F60008F5F8093A001FF91EF91BF91AF919F91EF
:102F70008F917F916F915F914F913F912F911F9111
:102F80000F91FF90EF900F900FBE0F901F9018952C
:102F9000CF93DF93CDB7DEB760970FB6F894DEBF5F
:102FA0000FBECDBF80915303909154039093910233
:102FB0008093900280919002909191026FE070E076
:102FC0000E948618AE014B5F5F4FDA01641BCE0191
:102FD0004096E62FEA0FFF27ED53FE4FE491ED9365
:102FE000A817B907B1F719821A821B821C822BE03D
:102FF0006EE089E00E946F0824E0AE014F5F5F4FF2
:103000006CE08EE00E946F08409190025091910216
:103010006CE08FE00E94F60C60960FB6F894DEBF6D
:103020000FBECDBFDF91CF910895FB019F01E894C2
:103030004230C4F04532B4F44A3029F497FB1EF410
:10304000909581959F4F642F77270E948618805D09
:103050008A330CF0895D8193CB010097A1F716F4B8
:103060005DE251931082C9010C946A18FA01CF9362
:10307000FF93EF93223044F1253234F5C22FE894C8
:10308000CA3049F497FB3EF4909580957095619510
:103090007F4F8F4F9F4F2C2F332744275527FF9368
:1030A000EF930E94AD18EF91FF91605D6A330CF0D1
:1030B000695D6193B901CA016050704080409040E1
:1030C00051F716F4CDE2C19310828F919F91CF9169
:1030D0000C946A18DC01FC0101900020E9F732979A
:1030E000AE17BF0730F47C916081708331976D9388
:1030F000F7CF0895991B79E004C0991F961708F03F
:10310000961B881F7A95C9F780950895AA1BBB1B4B
:1031100051E107C0AA1FBB1FA617B70710F0A61BD7
:10312000B70B881F991F5A95A9F780959095BC01F8
:10313000CD01089597FB092E07260AD077FD04D00C
:10314000E5DF06D000201AF4709561957F4F089551
:10315000F6F7909581959F4F0895A1E21A2EAA1B2C
:10316000BB1BFD010DC0AA1FBB1FEE1FFF1FA21737
:10317000B307E407F50720F0A21BB30BE40BF50B34
:10318000661F771F881F991F1A9469F760957095BD
:10319000809590959B01AC01BD01CF010895E19907
:1031A000FECFBFBBAEBBE09A11960DB20895E19978
:1031B000FECFBFBBAEBB0DBA11960FB6F894E29A24
:0631C000E19A0FBE089524
:1031C60001010300000A000044000023002300540C
:1031D600646653636552620051610050600050603E
:1031E6000051610052620053636554646667686902
:1031F6006A6B6B6A696867000000535363535341F7
:0E320600034E02870392020D0A0A1D0000000B
:00000001FF
